:1000000000000814000000000000000000000000D4
:1000100000000000000000000000000000000000E0
:1000200000000000000000000000000000000000D0
:1000300000000000000000000000000000000000C0
:1000400000000000000000000000000000000000B0
:02000004001FDB
:020000040020DA
:10000000A00038D50120B8D20000218A400000B4F9
:1000100003000014FF0365B2B20000940000001456
:10002000010000B9C0035FD6000040B9C0035FD62D
:10003000E0031EAAC0035FD6FE03002AC0035FD6FA
:10004000C0035FD600000000800A8A5220E4A77235
:10005000F6FFFF171F2003D5FD7BBFA9FD0300910D
:10006000800A8A5220E4A772F0FFFF97A0FF0736AC
:1000700000088A5220E4A772ECFFFF97001C00538F
:10008000FD7BC1A8C0035FD6FD7BBFA9800A8A5251
:10009000FD03009120E4A772E4FFFF970000001227
:1000A000FD7BC1A8C0035FD6FD7BBEA9FD03009107
:1000B000F30B00F9F303002A800A8A5220E4A772A6
:1000C000DAFFFF97A0FF2F36E103132A00088A52B8
:1000D000F30B40F920E4A772FD7BC2A8D1FFFF1704
:1000E000FD7BBFA9FD030091800A8A5220E4A7721C
:1000F000CEFFFF97A0FF4737FD7BC1A8C0035FD6A7
:10010000FD7BBEA9FD030091F35301A9F403002A6E
:1001100013048052731200518126D31A210C00124D
:1001200020DC001122C000113F2800714030801AED
:10013000DEFFFF9713FFFF35F35341A9FD7BC2A8F4
:1001400000048052D9FFFF17FD7BBFA9FD0300917A
:10015000ECFFFF97A0018052D4FFFF97FD7BC1A861
:1001600040018052D1FFFF17FD7BBEA980008A525B
:1001700021008052FD03009120E4A772F30B00F9E7
:10018000A8FFFF9780088A520100805220E4A772DE
:1001900013008052A3FFFF97000C8A520100805287
:1001A00020E4A7729FFFFF9780098A526100805266
:1001B00020E4A7729BFFFF97000A8A520100805239
:1001C00020E4A77297FFFF9780088A5201008052AF
:1001D00020E4A77293FFFF9700098A52C11880524A
:1001E00020E4A7728FFFFF97000D8A52C121805231
:1001F00020E4A7728BFFFF978000805200E4A77273
:100200008AFFFF9702640E12010084528000805220
:100210002100A07200E4A7724100012A81FFFF972C
:10022000801280520100805200E4A7727DFFFF9788
:10023000E003132A7306001182FFFF977F5A0271B1
:1002400081FFFF54001380520100985200E4A7720E
:100250001300805273FFFF97E003132A7306001107
:1002600078FFFF977F5A027181FFFF54001380527D
:100270000100805200E4A7726AFFFF97F30B40F978
:10028000000C8A5261008052FD7BC2A820E4A77254
:1002900064FFFF171F2003D5FD7BBEA9211FA052BD
:1002A000FD030091F30B00F91381965213E0A7723E
:1002B000E003132A5BFFFF97E003132A01408052FB
:1002C000F30B40F9211FA072FD7BC2A855FFFF1759
:1002D0000084965200E0A77254FFFF171F2003D539
:1002E000FD7BBBA9FD030091F35301A9F55B02A9B6
:1002F000F76303A9F96B04A99CFFFF971500009011
:1003000000CF8A52180080528046A2721700805295
:100310001A008052140080528CFFFF971600805202
:1003200044FFFF971300805288FFFF9739018052E6
:1003300020098052B58214915CFFFF97000980521A
:100340005AFFFF97A008805258FFFF97000B80527A
:1003500056FFFF97A001805254FFFF974001805243
:1003600052FFFF973DFFFF971FE8007140030054C5
:100370001F28007104184D7A6003005401781A1286
:100380003F1C017120080054610600513F5000716C
:10039000A8FEFF54A14A6138620000104188218BF9
:1003A00020001FD61F2003D51FE80071011C00513B
:1003B0002020801A7F560071000C00121710172A97
:1003C000C009005425FFFF971FE800717306001154
:1003D00001FDFF5433008052E3FFFF171F2003D5B8
:1003E0005A6F1C5313008052DFFFFF171F2003D5E5
:1003F000011C00511FE800712020801A73060011B3
:10040000000C001200101A2A1A3C0012D6FFFF1727
:100410001FE80071011C00512020801A000C0012FE
:100420001410142A941E00129F060071E005005457
:10043000940500349F0A007133039F1ACAFFFF1707
:10044000011C00511FE800712020801A1301805206
:10045000000C00121410142A941E0012C2FFFF1781
:10046000011C00511FE800712020801A7306001142
:10047000000C00121610162AD63E00125603162A39
:10048000B9FFFF171F2003D5A001805207FFFF9778
:10049000A005805205FFFF97A005805203FFFF973C
:1004A000A001805201FFFF9740018052FFFEFF979D
:1004B00040018052FDFEFF9700009052DFFEFF9743
:1004C00000008052F35341A9F55B42A9F76343A9A9
:1004D000F96B44A9FD7BC5A8C0035FD61F2003D5D7
:1004E000D3018052A0FFFF17E003182A13008052A7
:1004F00016FFFF979CFFFF17F70AC05AE003162A62
:10050000E103172AD802180BD3018052F802180B06
:10051000C4FEFF97D612001193FFFF171F2003D5CB
:1005200008082F2F2F2F271B131313130F0101015F
:080530000101010101000000BE
:00000001FF
